:0200000480007A
:100000006F008004732F2034930F80006308FF0378
:10001000930F90006304FF03930FB0006300FF038E
:10002000130F000063040F0067000F00732F2034CC
:1000300063540F006F00400093E19153171F0000BD
:1000400023223FFC6FF09FFF93000000130100008C
:10005000930100001302000093020000130300004C
:100060009303000013040000930400001305000034
:10007000930500001306000093060000130700001C
:100080009307000013080000930800001309000004
:1000900093090000130A0000930A0000130B0000EC
:1000A000930B0000130C0000930C0000130D0000D4
:1000B000930D0000130E0000930E0000130F0000BC
:1000C000930F0000732540F16310050097020000B4
:1000D000938202017390523073500018970200000F
:1000E00093824202739052309B021000939252030B
:1000F0009382F2FF7390023B9302F0017390023AF5
:100100007350403097020000938242017390523046
:10011000735020307350303093010000970200007C
:10012000938282EE73905230130510001315F5017F
:10013000635C05000F00F00F930110009308D005D9
:10014000130500007300000093020000638A0200A0
:1001500073905210B7B200009B82921073902230BD
:100160007350003097020000938242017390123462
:10017000732540F173002030B70001FF9B8000F031
:1001800013E7F0F09303F0F093012000631C771C59
:10019000B710F00F9B8000FF13E7000FB713F00FAD
:1001A0009B8303FF93013000631E771AB700FF00A3
:1001B0009B80F00F13E7F070B703FF009B83F37F82
:1001C000930140006310771AB7F00FF09B80F000A6
:1001D00013E7000FB7F30FF09B83F30F9301500069
:1001E00063127718B70001009B8010F09390000114
:1001F000938000F093E0000FB70301009B8313F09E
:1002000093930301938303FF93016000639C701435
:1002100013020000B710F00F9B8000FF13E7000FE0
:10022000130307001302120093022000E31452FE8E
:10023000B713F00F9B8303FF9301700063147312D5
:1002400013020000B700FF009B80F00F13E7F0706F
:100250001300000013030700130212009302200092
:10026000E31252FEB703FF009B83F37F93018000EC
:10027000631A730E13020000B7F00FF09B80F000BA
:1002800013E7000F13000000130000001303070022
:100290001302120093022000E31052FEB7F30FF096
:1002A0009B83F30F93019000631E730A13020000F7
:1002B000B710F00F9B8000FF13E7000F130212002E
:1002C00093022000E31652FEB713F00F9B8303FF47
:1002D0009301A0006318770813020000B700FF0025
:1002E0009B80F00F1300000013E7F0F013021200E0
:1002F00093022000E31452FE9303F0FF9301B00039
:100300006312770613020000B7F00FF09B80F00035
:10031000130000001300000013E7000F1302120087
:1003200093022000E31252FEB7F30FF09B83F30F0A
:100330009301C000631877029360000F9303000FCE
:100340009301D00063907002B700FF009B80F00F14
:1003500013E0F070930300009301E0006314700059
:10036000631030020F00F00F6380010093911100C1
:1003700093E111009308D00513850100730000007C
:100380000F00F00F930110009308D0051305000033
:1003900073000000731000C00000000000000000A7
:1003A000000000000000000000000000000000004D
:0C03B00000000000000000000000000041
:1010000000000000000000000000000000000000E0
:1010100000000000000000000000000000000000D0
:1010200000000000000000000000000000000000C0
:1010300000000000000000000000000000000000B0
:081040000000000000000000A8
:040000058000000077
:00000001FF
